:10000000830100308A001F28F00003088301A80044
:100010000A08A9008A01831203138C1E10281128D4
:1000200016281A08A000A301A30AA401031383122F
:1000300029088A0028088300F00E700E090020307D
:10004000840028302A2083010A128A111F2F0406F7
:100050008001840A0406031900342728831203133D
:10006000AA00AB1B3C282B1B44282B088A002A081B
:10007000AA0A0319AB0A820083132B1883172A08D4
:08008000AA0A84000008080030
:100D5A00831603131815193099001812831298175D
:100D6A008316981683121816031383120800831227
:100D7A000313A500C02E83160313981CC52EC62E76
:100D8A00C02E831203132508990003138312080047
:100D9A0083120313A600043083120313A5005330F1
:100DAA0083120313A700DA2EDA2E83120313A70B7A
:100DBA00DF2EE02ED92E83120313A50BE52EE62E85
:100DCA00D42E83120313A60BEB2EEC2ED02E031374
:100DDA008312080083120313A501082F8312031339
:100DEA0025082507AA002608AB002A080318AB0A1B
:100DFA000A128A112E200A128A110A128A11BC2694
:100E0A000A128A11A50A8312031325082507AA00C4
:100E1A002608AB002A080318AB0A0A128A112E20E8
:100E2A000A128A110038031D1B2F1C2FF32E0313DD
:100E3A00831208000A300A128A11CD260A128A1170
:100E4A000A128A11AD260A128A11063083169F00E9
:100E5A00EF309200871007110C3083129D000C307E
:100E6A0097008316091188100811881109100614B1
:100E7A00081405118910831212158316061283129B
:100E8A0088100811881506160B1383168C128B13FB
:100E9A00522F831203139B01950183120313081C1B
:100EAA00572F582F4E2FBE30831203139B00C83082
:100EBA00950083120313981C632F642F682F18124E
:100ECA00091418166B2F83120313091083120313C4
:100EDA008C1E702F712F822F1819742F752F792F4E
:100EEA0089141A08A000822F831203131808A2007B
:100EFA001A08A2001A08A000891083120313061CFC
:100F0A00872F882F952FA10A21080A3A031D8E2FB1
:100F1A008F2F942F831203139B0195018F2F982FE4
:100F2A0083120313A101D72FBE30831203139B0030
:100F3A0009110511C8309500F02F8C308312031364
:100F4A00950009110511C8309B00F02F64308312F7
:100F5A000313950009110511C8309B00F02F831265
:100F6A00031395010911051596309B00F02F8C305B
:100F7A00831203139B0009110511C8309500F02F45
:100F8A006430831203139B0009110511C8309500C0
:100F9A00F02F831203139B01091505119630950052
:100FAA00F02FF02F831203132008013A0319CE2FD2
:100FBA00033A0319C52F063A0319BC2F0C3A031931
:100FCA00992F183A0319A22F303A0319AB2F603A16
:100FDA000319B42FF02F831203131030860623034C
:100FEA002404031DF92FFA2FFC2FA301A4015E2F5D
:060FFA000A128A111F28F3
:02400E00393D3A
:00000001FF
